:103879000FC30FBF0FBB0FB60FB20FAC0FA70FA12E
:103889000F9B0F950F8E0F870F800F780F700F68A2
:103899000F5F0F550F4B0F410F360F2B0F1F0F12D5
:1038A9000F060EF80EEA0EDB0ECC0EBC0EAB0E9A0E
:1038B9000E880E750E620E4E0E390E240E0E0DF781
:1038C9000DDF0DC70DAE0D940D790D5E0D410D2463
:1038D9000D070CE80CC90CA90C890C680C460C23C3
:1038E9000C000BDC0BB80B930B6E0B480B210AFA7F
:1038F9000AD30AAC0A840A5B0A330A0A09E109B73E
:10390900098E0965093B091108E808BE0895086C84
:103919000842081907F107C807A0077807500729BF
:10392900070206DB06B5068F066A0645062105FD70
:1039390005DA05B70595057405530532051204F333
:1039490004D404B60498047B045F04430428040DDA
:1039590003F303DA03C103A90391037A0363034D54
:1039690003370322030E02F902E602D302C002AEB4
:10397900029C028B027A026A025A024B023C022D15
:10398900021F0211020301F601E901DD01D001C59F
:1039990001B901AE01A30198018E0184017A017177
:1039A9000168015F0156014D0145013D0135012EB7
:1039B9000126011F01180111010B010400FE00F885
:1039C90000F200EC00E600E100DC00D600D100CCFA
:1039D90000C800C300BE00BA00B600010C01010412
:1039E90002011E030A960401320503030600640757
:1039F900010108000009015A0E01010F000112001E
:103A09006413010114013C1501FA1664FA17FFFF4A
:103A19001D00072000072400022701012F013C3067
:103A2900010132010335FFFF3603073CFFFF3DFF6C
:103A3900FF0B0000180002191E461A01011B0101A3
:093A49002D32C82E0001FAFAFA30
:10004800900784E0FEA3E0FF7457BE0010D39F40E2
:100058000C9039E312001EE493F5998012900784FE
:10006800E0FEA3E0FF9039E312001EE493F59990B7
:10007800078412000E900784E0FEA3E0FF746F6F00
:100088004E700375130022900070E0B402087401EA
:10009800900070F0D20C900138E090002AF09001A6
:1000A80039E090002BF090013AE090002CF0A20A81
:1000B800B34016900138E0700C900139E07006905A
:1000C800013AE060028002C20A900138E0B4300FC1
:1000D800900139E0B4470890013AE0643B6002803F
:1000E80004D20B8002C20BE558B40102800302025D
:1000F80011900055E0F566900060E0F568900061A9
:10010800E0F569900072E0F56A900078E0900029C7
:10011800F090007AE0F56590007BE0F56790007E4E
:10012800E0F56490007FE0F56390008EE090004178
:10013800F090008FE0900042F0900090E090004333
:10014800F0900091E0900044F0900092E09000451B
:10015800F0900093E0900046F0900094E090004703
:10016800F0900095E0900048F0900097E090003300
:10017800F0900098E0900034F0900099E0900035FD
:10018800F090009AE0900036F0900077E0B4011704
:1001980090000A740FF0A374FFF090000CE4F0A331
:1001A800F07402900077F0900077E0B40359900063
:1001B8000CE0FEA3E0FF90000AE0FCA3E0FD1200C3
:1001C800037410123BB27408123BA4EF900026F09F
:1001D800EF700674FF900026F07400900077F0909E
:1001E800000BE0900027F090000AE0900028F090C3
:1001F8000026E0900787F0900027E0900788F090AD
:100208000028E0900789F0803F90007FE070067535
:100218005801756300A20AB3402E900138E090009F
:100228002AF0900139E090002BF090013AE090001C
:100238002CF090002AE0700C90002BE070069000E3
:100248002CE060028002C20AE5667003756602E56A
:100258006870037568027E837FC2E5668E048F0529
:10026800FF123B948C398D3AE56975F0FAA4FFAE1C
:10027800F0E5688E048F05FF123B948C3D8D3E900F
:10028800004DE0F560740190009CF0740190009DB1
:10029800F0740090009EF0740090009FF07400903D
:1002A80000A0F074009000A1F074009000A2F07417
:1002B800019000A3F074019000A4F074009000A5D0
:1002C800F074009000A6F074009000A7F0740090FD
:1002D80000A8F074009000A9F074019000AAF074CE
:1002E800019000ABF074009000ACF074009000AD89
:1002F800F074009000AEF074009000AFF0740090BD
:1003080000B0F07401900360F07401900361F07420
:1003180000900362F07400900363F074009003642B
:10032800F07400900365F07400900366F074009018
:1003380003A0F074019003A1F074009003A2F0747C
:10034800009003A3F074009003A4F074009003A538
:10035800F074009003A6F074009003E0F07400902D
:1003680003E1F074009003E2F074009003E3F0748A
:10037800009003E4F074009003E5F074009003E645
:10038800F07401900420F07400900421F07400903F
:100398000422F07400900423F07400900424F07494
:1003A80000900425F07400900426F022E5B554F777
:1003B800F5B5E5B554FDF5B5C2A2C2A1C292C20712
:1003C800E5B554FBF5B5755104E55104F5529000B7
:1003D8004DE0F560900025E4F0C209E5B554FEF55E
:1003E800B522750A00750900AE09AF0A7457BE0038
:1003F800039F50030204A79039E312001EE4939070
:10040800004C123BCA0FBF00010EE0FC9039E3120A
:10041800001EECFEE493FFEEC39F5026AE09AF0A20
:100428000FBF00010E9039E312001EAE09AF0AE4B7
:1004380093FC9039E312001EE49390004C123BCADF
:10044800ECF0AE09AF0A9039E312001EE493900075
:100458004C123BCAE0FC9039E512001EECFCE49318
:10046800FDECD39D40199039E512001EE493FC90F1
:1004780039E312001EE49390004C123BCAECF0AE34
:1004880009AF0A74022FFF50010E8E098F0A780AED
:10049800740126F6500418E436F640030203F022ED
:1004A800750A00750900AE09AF0A7418BE00039FEB
:1004B8005003020575903A3A12001EE49390004CDE
:1004C800123BCA0FBF00010EE0FC903A3A12001E20
:1004D800ECFEE493FFEEC39F5026AE09AF0A0FBFB0
:1004E80000010E903A3A12001EAE09AF0AE493FCDE
:1004F800903A3A12001EE49390004C123BCAECF07A
:10050800AE09AF0A903A3A12001EE49390004C12DA
:100518003BCAE0FC903A3C12001EECFCE493FDEC74
:10052800D39D4019903A3C12001EE493FC903A3A4D
:1005380012001EE49390004C123BCAECF0AE09AFD7
:100548000A74126F4E7006750A18750900AE09AF65
:100558000A74022FFF50010E8E098F0A780A74015F
:1005680026F6500418E436F640030204AE22054D80
:1005780022054C22054EC2CF2290F800E49364066F
:10058800600280FE75840175A70075FF809007865C
:10059800E4F075C91075A70F75A1C775A70075D9BF
:1005A8000075CEFF75A70F75F1FE75F2FF75F3376D
:1005B80075F47875A4BA75A5FF75A60775AE0075AC
:1005C800AFFF75D48175D5FF75D6FF75D7FFC29675
:1005D800C295C2A0C297E5B554BFF5B5E5B554DFDD
:1005E800F5B5E5B554EFF5B5E5B5547FF5B5E5B521
:1005F80054F7F5B5E5B554FDF5B575A70075A20135
:1006080075A14775F80975BC0175BE0475BD6C7593
:10061800BE0775BDA075BE0875BD0175BC0075BB6C
:100628001875BC2075BA0875E88075D11375A70FC1
:1006380075E10575E20075C7407597007597807478
:100648000A123B847597C0E5975420700280F875AC
:100658008F0275A700D2AF75980075A90C75A70F02
:1006680075AB4375ADFB75AC1E75A7007589117523
:100678008E00758C00758A00D2A9D28C758D007594
:100688008B00D2ABD28E75CD0075CC0075CA0075C3
:10069800CB00D2ADC2CFD2CA7591047592007593C2
:1006A800CD75EF0675D94075CF01900784E4F0A3A6
:1006B800F0751300751400C299D20A74C8F518753C
:1006C80017001221A275A70FE5FB90001AF0E5FAB2
:1006D80090001BF0E5F990001CF075A70090F80059
:1006E800E493F5081222D9122813900787E09000A6
:1006F80026F0900788E0900027F0900789E09000A6
:1007080028F090078AE0900029F090078BE0F566C2
:1007180090078CE0F56890078DE0F56990078EE00A
:10072800F56A90078FE0F565900790E0F567900708
:1007380091E0F564900792E0F563900793E09000EC
:100748002AF0900794E090002BF0900795E0900035
:100758002CF0900796E0900041F0900797E0900009
:1007680042F0900798E0900043F0900799E09000DD
:1007780044F090079AE0900045F090079BE09000C5
:1007880046F090079CE0900047F090079DE09000AD
:1007980048F090079EE0900033F090079FE09000AB
:1007A80034F09007A0E0900035F09007A1E09000A9
:1007B80036F07400900080F0900138E0700C9001E1
:1007C80039E0700690013AE060028004C20A8002B3
:1007D800D20A90F807E493900021F0900021E044B9
:1007E8000A900021F0900021E054FE900021F0745E
:1007F80006900012F07402900013F090F802E4934F
:10080800900014F07403900015F07403900016F033
:100818007411900017F07405900018F0740490009B
:1008280019F090F804E49390001DF0740090001EF5
:10083800F090F805E49390001FF090F806E4939088
:100848000020F074FF900022F0744A900123F074A5
:1008580061900124F07474900125F074639001266E
:10086800F0746F900127F07420900128F074529072
:100878000129F0744590012AF0743490012BF0742A
:100888002090012CF0742090012DF0744F90012ECF
:10089800F0744590012FF0744D900130F074209061
:1008A8000131F0900078E0D3940140067400900084
:1008B80078F075580175590112008F1203EA120475
:1008C800A81221CEE5B554FEF5B5900025E4F090C8
:1008D8000784E4F0A3F075240075230075480075BB
:1008E8002A00752900754900753200753100754A6E
:1008F80000755400755500755A00755104755201FC
:1009080075343C753300757000756F007571CD7561
:1009180056007557007543007544007545007546C7
:1009280000755B0075470075420075410090000630
:10093800E4F0A3F0900008E4F0A3F0755E00755FA2
:100948000090000E74FDF0A374E8F0900023E4F02A
:100958007464900024F0C200D201C202D203754D23
:1009680000756D00C294C293C287C290C29174038D
:1009780090004BF0C20C7E017F00900028E0123BF3
:10098800B2900027E02FFF50010E90000AEEF0A36E
:10099800EFF0900026E0700674FF900026F09000BB
:1009A8000AE0FEA3E0FFEFD394FFEE940F40079018
:1009B800000AE4F0A3F0740090006FF07400900057
:1009C80077F07400900080F0740090008BF0740051
:1009D8009000B2F0E5677003756704743A90074CAD
:1009E800F074FD90074DF09003D2E0900412F0D21D
:1009F800B0D2B7D2A7D2A6D2B1D2A3C207A2B6B3F9
:100A08009204A2B3B39205A2A5920DA2A4920ED20B
:100A18009CD2EC75CF01A298B34005C298122B77EF
:100A2800E5136006A299B3B340028005C29912305B
:100A3800EDE51464016005E514B4040280D5E54DC4
:100A4800D39405400CE55AC394C85002055A754D15
:100A580000E571C394F0501A786F12003FAE6FAF83
:100A680070EFD394E8EE9403400805717570007533
:100A78006F00C28E7E047F00E54C123BB2E58D7597
:100A8800F004A4FDACF0EF2DFDEE3CFCE58B75F019
:100A98004084FF7E00ED2FFFEC3EFE8E258F26D290
:100AA8008EA2B6300401B35003020BE1A2B63004A3
:100AB80001B35003020BE1A2B6405A0554E5B54410
:100AC80001F5B5900024E4F0E554D3956640447CE4
:100AD800837DC2123A528E238F24E5482FFF50019E
:100AE8000E7401123BA48E238F248524487554016B
:100AF800C28E758D00758B00754C00D28E7403BE46
:100B080000039F50069000257401F0E543B40603E6
:100B1800754300D204A2B6B35003020BE1C204909D
:100B28000069E0601812322EA200B34008E5B5440F
:100B380008F5B58006E5B554F7F5B58002C2009012
:100B4800006CE06018123383A202B34008E5B54494
:100B580002F5B58006E5B554FDF5B58006E5B55452
:100B6800FDF5B5A207B34004D2878002C287900082
:100B780057E06004D2908002C29090004AE0B4012D
:100B880004D2948002C294900049E0B40104D29344
:100B98008002C293A209B34004D2918002C291900C
:100BA8000018E0FE900014E0C39E4009900014E095
:100BB800D39408400974FB900023F01203B490000A
:100BC8001DE0601590001DE0FE900017E06E6009C2
:100BD80074FE900023F01203B4C2CA7E017F00E5C0
:100BE8004E123BB2E5CD2FFF50010E8E278F28D233
:100BF800CAE565B4014890000EE0FCA3E0FDEFC330
:100C08009DEE9C4039B208E52A45296013A208B335
:100C18004008E5B54404F5B58006E5B554FBF5B5DF
:100C280090000EE0FEA3E0FF900010E0FCA3E0FDC2
:100C3800EF2DFDEE3CFC90000EECF0A3EDF0A2B31E
:100C4800300501B35003020D26A2B3300501B3509D
:100C580003020D26A2B35003020D1F0555E5B54446
:100C680001F5B5900024E4F0E555D39568500302EA
:100C78000D1D7CEA7D60AE27AF28123A528E298F6F
:100C88002AE569123BB274FF8E048F05FF123B946C
:100C98008C298D2AE5492DFD50010C74018C068D97
:100CA80007123BA48E298F2A852A49A209B3401529
:100CB8007464123BB2900065E08E048F05FF123B0E
:100CC800948C298D2A75550190000EE0FEA3E0FF53
:100CD800AC27AD2812000390000EEEF0A3EFF0E56C
:100CE80067FF123B94740AFF123B94900079E08CE2
:100CF800068D07123BB274148E048F05FF123B94C5
:100D0800900010ECF0A3EDF0C2CA75CD0075CC00D0
:100D1800754E00D2CAD205A2B3B34002C2059000F4
:100D280025E0B40107E556C394064003021366E5BF
:100D38006D902154F8282873900057E0C39402401E
:100D480003020E94E551D394015003020E94E55129
:100D580075F040A4FFAEF090031012001EE0C3959A
:100D6800455018E55175F040A4FFAEF090030F12FE
:100D7800001EE0F52E752D00020E94E55175F04029
:100D8800A4FFAEF090030E12001EE0C39545400389
:100D9800020E30E55175F040A4FFAEF090030F123B
:100DA800001EE55175F040A4FFAEF0E0FC90030D85
:100DB80012001EECFEE0FFEEC39FFEE5518E0475A7
:100DC800F040A4FFAEF090030E12001EE0F40425DC
:100DD800458C0088F0A4FFAEF0E5518F048E0575B0
:100DE800F040A4FFAEF090031012001EE55175F01C
:100DF80040A4FFAEF0E0FA90030E12001EEAFEE0F7
:100E0800FFEEC39FFECDCCCD8E07123B94E5517506
:100E1800F040A4FFAEF090030D12001EE02DFD502F
:100E2800010C8C2D8D2E8064E55175F040A4FFAE29
:100E3800F090030D12001EE55175F040A4FFAEF0CE
:100E4800E0FC90030C12001EECFEE0FFEEC39F8551
:100E580045F0A4FFAEF0E5518F048E0575F040A46F
:100E6800FFAEF090030E12001EE0FECDCCCD8E0733
:100E7800123B94E55175F040A4FFAEF090030C12BC
:100E8800001EE02DFD50010C8C2D8D2E756D01027C
:100E98001366900057E0C394024003021048900084
:100EA8004DE0D395515003020FF0E55175F040A481
:100EB800FFAEF090031612001EE0C395455018E5EA
:100EC8005175F040A4FFAEF090031512001EE0F536
:100ED8002C752B00020FF0E55175F040A4FFAEF021
:100EE80090031412001EE0C395454003020F8CE5E1
:100EF8005175F040A4FFAEF090031512001EE551A5
:100F080075F040A4FFAEF0E0FC90031312001EEC55
:100F1800FEE0FFEEC39FFEE5518E0475F040A4FF8E
:100F2800AEF090031412001EE0F40425458C0088EE
:100F3800F0A4FFAEF0E5518F048E0575F040A4FFD4
:100F4800AEF090031612001EE55175F040A4FFAEF6
:100F5800F0E0FA90031412001EEAFEE0FFEEC39FD1
:100F6800FECDCCCD8E07123B94E55175F040A4FF21
:100F7800AEF090031312001EE02DFD50010C8C2BD7
:100F88008D2C8064E55175F040A4FFAEF0900313FA
:100F980012001EE55175F040A4FFAEF0E0FC90038E
:100FA8001212001EECFEE0FFEEC39F8545F0A4FF81
:100FB800AEF0E5518F048E0575F040A4FFAEF090B9
:100FC800031412001EE0FECDCCCD8E07123B94E533
:100FD8005175F040A4FFAEF090031212001EE02DF0
:100FE800FD50010C8C2B8D2CE551B40123E560D309
:100FF8009401401CE55604D395514014E545C3942B
:1010080005500D90035DE0A829B80006952A400216
:101018008003755102E551B5602290004DE0D395EB
:10102800514019E55175F040A4FFAEF09003151238
:10103800001EE0A823B8000695244002800205603F
:10104800756D02021366900057E0B4022AE55175E7
:10105800F040A4FFAEF090031512001EE0F52C75C9
:101068002B00E55175F040A4FFAEF090030C120080
:101078001EE0F52E752D00900057E0B4030F900088
:101088004FE0F52C752B00752E00752D00756D033E
:10109800021366E55175F040A4FFAEF090031E12EE
:1010A800001EE0C3955A4003021170900049E07099
:1010B80036E551D394014029AE23AF24AC2DAD2E93
:1010C800EDD39FEC9E401AE55175F040A4FFAEF0B9
:1010D80090031C12001EE0A829B80005D3952A50D9
:1010E80002800215518034E551D394024029AE2381
:1010F800AF24AC2DAD2EEDD39FEC9E401AE5517573
:10110800F040A4FFAEF090031C12001EE0A829B81E
:101118000005D3952A500280021551E551B5523782
:10112800E551C395605030E55604D395514028AE3B
:1011380023AF24AC2BAD2CEFD39DEE9C4019E55189
:1011480075F040A4FFAEF090031D12001EE0A82920
:10115800B80006952A400280020551C292E5516501
:10116800526005C207755A00756D04021366E55191
:1011780075F040A4FFAEF090031812001EE0B40111
:1011880017E55175F040A4FFAEF090031E12001E43
:10119800E0240AC3955A4003021246753064752F3D
:1011A80000A207B3500B90005EE02405C3954540AC
:1011B80003021246E55175F040A4FFAEF090031B00
:1011C80012001EE0C395454064E55175F040A4FF48
:1011D800AEF090031A12001EE55175F040A4FFAE60
:1011E800F0E0FC90031912001EECFEE0FFEEC39F36
:1011F8008545F0A4FFAEF0E5518F048E0575F040EB
:10120800A4FFAEF090031B12001EE0FECDCCCD8EE5
:1012180007123B94E55175F040A4FFAEF090031916
:1012280012001EE02DFD50010C8C2F8D30AE23AF27
:1012380024AC2FAD30EFD39DEE9C4002D207756DE4
:1012480005021366E551B40109900057E0C3940202
:10125800400302131C900356E0D395455003021334
:101268001A900354E0C395455040900355E0FE9012
:101278000353E0F4042EFE900354E0F40425458E55
:101288000088F0A4FFAEF0900356E0FC900354E011
:10129800F4042C8E048F05FF123B94900353E02D29
:1012A800FD50010C8C2B8D2C802C900353E0FE906C
:1012B8000352E0F4042E8545F0A4FFAEF0900354E9
:1012C800E08E048F05FF123B94900352E02DFD50F1
:1012D800010C8C2B8D2CE551C395605030E55604DC
:1012E800D395514028AE23AF24AC2BAD2CEFD39D22
:1012F800EE9C4019E55175F040A4FFAEF090031D37
:1013080012001EE0A829B80006952A40028003753D
:101318005102802AE551D39560401AE55175F04095
:10132800A4FFAEF090031C12001EE0A829B8000527
:10133800D3952A500280071551C207755A009000AC
:1013480049E0B40106E55164016002800375510269
:0E135800E55165526005C207755A00756D00BB
:10215400020D40020E9A02104E02109B02117602EA
:02216400124C1B
:1013660090004EE02402A823B80007D3952440023B
:10137600C207900025E0B40109900057E0C394032A
:1013860040030214EE900049E0600302143DE5516B
:10139600D394014034E55175F040A4FFAEF09003BC
:1013A6001212001EE0A823B8001FD39524401AE5A8
:1013B6005175F040A4FFAEF090031D12001EE0A888
:1013C60029B80005D3952A500280021551E551D35C
:1013D6009401402FE55175F040A4FFAEF090031044
:1013E60012001EE0C39545501AE55175F040A4FF62
:1013F600AEF090031C12001EE0A829B80005D39594
:101406002A500280021551E551D394014022E55637
:1014160004C39551501AE55175F040A4FFAEF09003
:10142600031C12001EE0A829B80005D3952A500215
:10143600800215510214E3E551D394024034E5517C
:1014460075F040A4FFAEF090031212001EE0A82330
:10145600B8001FD39524401AE55175F040A4FFAE9D
:10146600F090031D12001EE0A829B80005D3952AA6
:10147600500280021551E551D39402402FE5517573
:10148600F040A4FFAEF090031012001EE0C3954595
:10149600501AE55175F040A4FFAEF090031C1200FF
:1014A6001EE0A829B80005D3952A500280021551DE
:1014B600E551D394024022E55604C39551501AE5EE
:1014C6005175F040A4FFAEF090031C12001EE0A878
:1014D60029B80005D3952A500280021551E55165B9
:1014E600526005C207755A0090005EE0D3954550DC
:1014F60009900052E0C395455002C207A2A5300DDF
:1015060001B3404BA2A5400D90004A7401F07560EE
:1015160004D294D20DA2A5B3403590004AE4F075EA
:101526006003C294E551B4041AE55175F040A4FF76
:10153600AEF090031C12001EE0A829B80005D39552
:101546002A50028008755103C207755A00C20DA2BF
:10155600A4300E01B3401CA2A4400A9000497401B5
:10156600F0D293D20EA2A4B34009900049E4F0C28F
:1015760093C20EE55865596006900080E06003024C
:101586001701C29C751400751300C2CAE558902154
:1015960066F82828738012122813800D1228EC8012
:0915A600081229C58003122A9ED7
:0F21660002159B02159D0215A20215A70215ACCA
:1015AF00900029E0900078F0E566900055F0E5682E
:1015BF00900060F0E569900061F0E56A900072F0CC
:1015CF00E56590007AF0E56790007BF0E5649000A8
:1015DF007EF0E56390007FF090002AE0900138F0F4
:1015EF0090002BE0900139F090002CE090013AF040
:1015FF00900041E090008EF0900042E090008FF05C
:10160F00900043E0900090F0900044E0900091F043
:10161F00900045E0900092F0900046E0900093F02B
:10162F00900047E0900094F0900048E0900095F013
:10163F00900033E0900097F0900034E0900098F025
:10164F00900035E0900099F0900036E090009AF00D
:10165F007400900080F0744A900123F0746190013F
:10166F0024F07474900125F07463900126F0746F68
:10167F00900127F07420900128F07452900129F006
:10168F00744590012AF0743490012BF0742090016E
:10169F002CF0742090012DF0744F90012EF07445B2
:1016AF0090012FF0744D900130F07420900131F0C3
:1016BF009003D2E0900412F0743A90074CF074FD4E
:1016CF0090074DF012008F900004E4F0A3F090000B
:1016DF00067475F0A37430F09000087475F0A3745D
:1016EF0030F0855859D2CA754C00D29C741B9000AB
:1016FF0023F0E556C394065005E551B55202804ECE
:10170F00C207E55175F040A4FFAEF0900320120020
:10171F001EE030E003D38001C39296E55175F0408F
:10172F00A4FFAEF090032112001EE030E003D3803F
:10173F0001C39295855152AE29AF2A7405BE00039D
:10174F009F5007E545D3940550028002D292E5568B
:10175F00D394055003021826C207E551D3940140D4
:10176F0059E55175F040A4FFAEF090031C12001E16
:10177F00E0A829B80007D3952A40021551E5516515
:10178F00526035E55175F040A4FFAEF09003201282
:10179F00001EE030E003D38001C39296E55175F04F
:1017AF0040A4FFAEF090032112001EE030E003D3FF
:1017BF008001C39295855152805DE556B4061A900B
:1017CF0000AAE030E003D38001C392969000ABE013
:1017DF0030E003D38001C39295E556B4071A900009
:1017EF00A3E030E003D38001C392969000A4E030D1
:1017FF00E003D38001C39295E556B4081A90009C7C
:10180F00E030E003D38001C3929690009DE030E07A
:10181F0003D38001C39295900070E06058E5457541
:10182F00F00284FF7E0090014C12001EE0F55CE593
:10183F004775F00A84FF7E0090024C12001EE0F5FF
:10184F005DE55C255DD39464400BE55C255DC39439
:10185F0064F55C8003755C00E55C75F00284FF7EC7
:10186F00008F5CEFC394335007EF24CDF55C8003FA
:10187F00755CFF801CE54575F00284FF7E009001CA
:10188F004C12001EE075F00284FF7E00EF24CDF5B0
:10189F005CE595C3955C4004C2A28002D2A2A20768
:1018AF00B34005E556B407037571CDE595C3957142
:1018BF004004C2A18002D2A1E543C39406400302B3
:1018CF001F45A2EDB35003021F45C2EDE543600370
:1018DF00021A2C7E017F00E5BE123BB2E5BD2FFF41
:1018EF0050010E900000EEF0A3EFF0900029E0B44D
:1018FF0001177E0F7FFF900000E0FCA3E0FD1200B8
:10190F0003900000EEF0A3EFF0900077E0B4025BDD
:10191F00900000E0FEA3E0FF90000AE0FCA3E0FDD2
:10192F00EDD39FEC9E400F900000E0F8A3E09000F5
:10193F000AC8F0A3C8F0900000E0FEA3E0FF9000FB
:10194F000CE0FCA3E0FDEFD39DEE9C400F90000058
:10195F00E0F8A3E090000CC8F0A3C8F0900000E0FE
:10196F00FEA3E0FF7404123BA48F44900077E07055
:10197F0060900000E0FEA3E0FF90000AE0FCA3E00F
:10198F00FDEFD39DEE9C400D120003900000EEF092
:10199F00A3EFF08007900000E4F0A3F0900000E0C8
:1019AF00FEA3E0FF7410123BB2900026E08E048F6E
:1019BF0005FF123B94900000ECF0A3EDF07400D300
:1019CF009D74019C4008900001E0F544800375442C
:1019DF00FFE54475F00AA4FFAEF074198E048F056D
:1019EF00FF123B948D45ED2532FFAE3150010E7441
:1019FF0001123BA48F45854532753100EFD39462B8
:101A0F004003754562900070E064016006900064C9
:101A1F00E060028005754301800375BB17E543B491
:101A2F0001028003021B1C7E017F00E5BE123BB248
:101A3F00E5BD2FFF50010E900000EEF0A3EFF090E8
:101A4F000070E0B4017EE53445336025AC33AD342E
:101A5F001DBDFF011C8F028E038C068D07903879F8
:101A6F0012002EE493FE740193FFEFC39AEE9B4096
:101A7F000280057833123BDCAE33AF3474B3BE0053
:101A8F0025D39F4021900000E0FCA3E0FD0FBF0095
:101A9F00010E90387912002EE493FE740193FFED3E
:101AAF00C39FEC9E40028005783312003FAE33AFE8
:101ABF0034E56A123BB274648E048F05FF123B94B7
:101ACF008D478033900064E0602D900000E0FEA30E
:101ADF00E0FFEFD39400EE9408400F900064E0B461
:101AEF000104C2098002D209800D900064E0B401A4
:101AFF0004D2098002C209900070E064026006906F
:101B0F000064E0600575BB168003754302E543B4BE
:101B1F0002028003021C0A7E017F00E5BE123BB267
:101B2F00E5BD2FFF50010E900000EEF0A3EFF090F7
:101B3F000070E0B4027EE53445336025AC33AD343C
:101B4F001DBDFF011C8F028E038C068D0790370F72
:101B5F0012002EE493FE740193FFEFC39AEE9B40A5
:101B6F000280057833123BDCAE33AF3474B3BE0062
:101B7F0025D39F4021900000E0FCA3E0FD0FBF00A4
:101B8F00010E90370F12002EE493FE740193FFEDB8
:101B9F00C39FEC9E40028005783312003FAE33AFF7
:101BAF0034E56A123BB274648E048F05FF123B94C6
:101BBF008D478033900064E0602D900000E0FEA31D
:101BCF00E0FFEFD39400EE9408400F900064E0B470
:101BDF000104C2098002D209800D900064E0B401B3
:101BEF0004D2098002C209900070E07003754700AB
:101BFF00900064E07002C20975BB1FE543B4034552
:101C0F007E017F00E5BE123BB2E5BD2FFF50010EF6
:101C1F00900000EEF0A3EFF07409123BB274E68E61
:101C2F00048F05FF123B948C418D42E54A2DFD50E8
:101C3F00010C74018C068D07123BA48E418F4285D7
:101C4F00424A75BB19E543B404028003021E067EA7
:101C5F00017F00E5BE123BB2E5BD2FFF50010E9094
:101C6F000000EEF0A3EFF07404123BA48F4BE56479
:101C7F00B401028003021D3F756B00756B00E56BAD
:101C8F00D394074003021D2CE56B900041123BCA11
:101C9F00E0D3954B501AE56B900041123BCAE0F42C
:101CAF0004254BFEE56B900037123BCAEEF0801710
:101CBF00E56B900041123BCAE0C3954BFEE56B907C
:101CCF000037123BCAEEF0E56BC394044009900055
:101CDF0082E0C3956B503BE56B6029E56B90003755
:101CEF00123BCAFEE0FFEE90003FE0D39F4013E5AA
:101CFF006B900037123BCAE090003FF0E56B90000D
:101D0F0040F0800E900037E090003FF0740090009C
:101D1F0040F0786B740126F64003021C8D90004052
:101D2F00E0F4042408F556E556D394054002C29218
:101D3F00E564D39401402FE54BD3946E4004D20F4A
:101D4F008002C20F755605E564B40205A20FB340B9
:101D5F00028003755607E564B40306A20FB3B340C0
:101D6F00028003755607E55765566008E55104F57F
:101D7F0052855657E556902175F82828738049D219
:101D8F00A08045E544C394105004D2A08002C2A0A5
:101D9F008036E551C394045007E544C394104002C4
:101DAF008004D2A08002C2A0801E801CE551C39483
:101DBF00045007E544C3941040028004D2A080026F
:081DCF00C2A080048002800024
:10217500021D8C021D8E021D92021DA1021DB902B7
:0B2185001DBB021DD3021DD5021DD79B
:101DD700E556B40708E5B54480F5B58006E5B55482
:101DE7007FF5B5E55664066005E556B40808E5B520
:101DF7004410F5B58006E5B554EFF5B575BB13E5A9
:101E070043B405028003021F417E017F00E5BE1235
:101E17003BB2E5BD2FFF50010E900000EEF0A3EF9F
:101E2700F07404123BA48F46E563B40202800302F8
:101E37001F3E900000E0FCA3E0FDEDD3946DEC9411
:101E4700074029EDD3947FEC940D4005756C058010
:101E570019900000E0FEA3E0FF747FD39F74099EF2
:101E67004005756C038003756C04802F900000E0BB
:101E7700FEA3E0FF7445D39F74059E4005756C0073
:101E87008019900000E0FEA3E0FFEFD3944CEE949E
:101E9700064005756C028003756C0190004AE4F0FA
:101EA700900049E4F0755801E56C902190F82828D6
:101EB7007390004A7401F09000497401F0802090FB
:101EC700004A7401F0755802801590004A7401F0B9
:0F1ED700800D9000497401F0800575580280005D
:10219000021EB8021EC6021ED1021ED9021EE10294
:0221A0001EE639
:101EE60090004AE0FE90004BE06E601E900057E0C6
:101EF600B4010F90004AE0B40105756004800375D3
:101F0600600390004AE090004BF0E560B4031FE5E3
:101F160051B4041AE55175F040A4FFAEF090031CCD
:101F260012001EE0A829B80005D3952A50028008A1
:101F3600755103C207755A0075BB180543D2ECE507
:101F46005ED39404500302202D75CF01C2A2AE3594
:101F5600AF367488D39F74139E4005A2A5B3401470
:101F6600AE35AF367488D39F74139E4005A2A4B3D2
:101F760040028048783512003FAE35AF36EFB48860
:101F86003BEEB41337A2A5B3500990004DE0D395AC
:101F9600515002800405518011A2A5B3500890004B
:101FA6004DE0655160028002D207A2A4B35007E556
:101FB60051D39401500280041551C207A2A5B3B3B0
:101FC6005006A2A4B3B340028006753600753500EC
:101FD600E55165526035E55175F040A4FFAEF090CD
:101FE600032012001EE030E003D38001C39296E581
:101FF6005175F040A4FFAEF090032112001EE030B0
:10200600E003D38001C39295855152A2074005751E
:1020160071CD80037571FFE595C395714004C2A12A
:102026008002D2A1021F4FAE25AF26EFD39420EE39
:10203600944E50030221281203B4C28E758D00758A
:102046008B00754C00D28EC207757000756F0075D7
:1020560071CD755104752400752300755400755AA9
:1020660000C287900057E06004D2908002C2909030
:10207600004AE0B40104D2948002C294900049E080
:10208600B40104D2938002C293A209B34004D29150
:102096008002C291900069E0601812322EA200B34D
:1020A6004008E5B54408F5B58006E5B554F7F5B53D
:1020B6008002C20090006CE06018123383A202B363
:1020C6004008E5B54402F5B58006E5B554FDF5B51D
:1020D6008006E5B554FDF5B590000E74FDF0A374C9
:1020E600E8F0E543B40603754300900025E4F07577
:1020F6002600752500758D00758B00754C009000C7
:1021060024E0C394035008900024E004F080067491
:1021160003900024F0900024E0B40306E5B554FED5
:10212600F5B5AE27AF28EFD39410EE9427401CC226
:10213600CA75CD0075CC00752800752700D2CA7502
:0E2146004E00752A00752900755500020A1B0F
:1035350000000100013201640196019602000212A9
:1035450002240200020003000340038003C00400BC
:103555000440048004C005000600060006000600BD
:10356500060006000600060000FF01310163019513
:1035750001FF01FF0211022302FF02FF02FF033FC9
:10358500037F03BF03FF043F047F04BF04FF05FF60
:1035950006FF06FF06FF06FF06FF06FF06FF06FFFE
:1035A5000FAA0FA50F9F0F9A0F940F8D0F870F80EE
:1035B5000F780F710F680F600F570F4E0F450F3BB8
:1035C5000F300F250F1A0F0E0F020EF50EE80EDB4A
:1035D5000ECC0EBE0EAE0E9F0E8E0E7D0E6C0E5ACE
:1035E5000E470E340E200E0C0DF70DE20DCB0DB56A
:1035F5000D9D0D850D6D0D540D3A0D200D050CE934
:103605000CCE0CB10C940C760C580C3A0C1B0BFB25
:103615000BDB0BBB0B9A0B790B570B350B130AF115
:103625000ACE0AAB0A870A640A400A1C09F809D4BB
:1036350009B0098C09670943091F08FB08D608B2B8
:10364500088E086A0846082307FF07DC07B90796AE
:1036550007730751072F070D06EC06CA06AA068948
:1036650006690649062A060A05EC05CD05B0059248
:1036750005750558053C0520050504EA04CF04B584
:10368500049C04820469045104390422040B03F4E4
:1036950003DE03C803B2039D038903750361034D6C
:1036A500033B03280316030402F202E102D102C020
:1036B50002B002A00291028202730265025702491A
:1036C500023C022F02220216020901FD01F201E667
:1036D50001DB01D001C601BB01B101A7019D019428
:1036E500018B018201790170016801600158015067
:1036F5000148014101390132012B0125011E011843
:103705000111010B010500FF00FA0FA60FA00F998B
:103715000F920F8B0F840F7C0F740F6B0F620F5876
:103725000F4E0F430F380F2C0F1F0F120F050EF7FB
:103735000EE80ED80EC80EB70EA50E930E800E6CB1
:103745000E580E420E2C0E150DFD0DE40DCB0DB1D0
:103755000D950D790D5D0D3F0D200D010CE10CC092
:103765000C9E0C7C0C590C350C100BEA0BC40B9EF3
:103775000B760B4F0B260AFD0AD40AAA0A800A55B6
:103785000A2A09FF09D409A8097C0950092508F95D
:1037950008CD08A10875084A081E07F307C8079D44
:1037A50007730749072006F706CE06A6067E0657C5
:1037B5000630060A05E405BF059B05770554053265
:1037C500051004EF04CE04AE048F047104530435D0
:1037D500041903FD03E203C703AD0394037B0363ED
:1037E500034B0334031E030802F302DE02CA02B6CA
:1037F50002A30291027F026D025C024C023C022C84
:10380500021D020E020001F201E401D701CA01BE48
:1038150001B101A6019A018F0185017A0170016646
:10382500015D0153014A014101390131012901219C
:1038350001190112010B010400FD00F700F000EA77
:1038450000E400DE00D900D300CE00C900C400BFEB
:1038550000BA00B500B100AD00A800A400A0009C0E
:10386500009900950091008E008A008700840081F0
:04387500007E007B56
:1021A200751A00751900AE19AF1AAC17AD18EDC348
:1021B2009FEC9E401674FF123B8475CF01781A740F
:1021C2000126F6500418E436F650DB22900784E428
:1021D200F0A3F0751000750F00751300751400C29E
:1021E20010D21122C2AF75D900758F0375B7A575CC
:1021F200B7F190F800E4F0758F0175B7A575B7F1E6
:10220200E50890F800F075B7A575B7F190F801E40C
:10221200F075B7A575B7F190079BE090F802F075DD
:10222200B7A575B7F190079FE090F803F075B7A5D1
:1022320075B7F190079CE090F804F075B7A575B7F3
:10224200F190079DE090F805F075B7A575B7F1908C
:10225200079EE090F806F075B7A575B7F19007A054
:10226200E090F807F0758F0075D940D2AF22900741
:1022720086E0B4AB61C2AF75D90075B62275F5229E
:10228200758F0375B7A575B7F1740090F600F075F8
:102292008F01750A00750900AE09AF0A7413BE00FA
:1022A200279F402475B7A575B7F190078712001EC6
:1022B200E0FC90F60012001EECF0780A740126F69B
:1022C200500418E436F650D0758F0075F51175B6C6
:1022D2002075D940D2AF22C2AF75D90075F52275EB
:1022E2000A00750900AE09AF0A7413BE00229F40AE
:1022F2001F90F60012001EE493FC90078712001E46
:10230200ECF0780A740126F6500418E436F650D53B
:1023120075F51175D940D2AF22900786E0B4AA02B2
:102322008003022458C2AF75D90075B62275F52212
:10233200758F0375B7A575B7F1740090EE00F0754F
:10234200B7A575B7F1740090F000F075B7A575B731
:10235200F1740090F200F075B7A575B7F1740090B2
:10236200F400F0758F01750A00750900AE09AF0A15
:1023720074FFC39F74019E402475B7A575B7F19091
:10238200004C12001EE0FC90EE0012001EECF078F1
:102392000A740126F6500418E436F650CF750A0086
:1023A200750900AE09AF0A74FFC39F74019E4024F1
:1023B20075B7A575B7F190024C12001EE0FC90F0C3
:1023C2000012001EECF0780A740126F6500418E49C
:1023D20036F650CF750A00750900AE09AF0A74FFD0
:1023E200C39F74019E402475B7A575B7F190044C44
:1023F20012001EE0FC90F20012001EECF0780A744B
:102402000126F6500418E436F650CF750A00750915
:1024120000AE09AF0A74FFC39F74019E402475B7D2
:10242200A575B7F190064C12001EE0FC90F4001264
:10243200001EECF0780A740126F6500418E436F611
:1024420050CF758F0075F51175B62075D940D2AF92
:10245200743A90074CF022900786E0B4AA028003F7
:10246200022596C2AF75D90075B62275F522758F11
:102472000375B7A575B7F1740090E600F075B7A5BE
:1024820075B7F1740090E800F075B7A575B7F174EF
:102492000090EA00F075B7A575B7F1740090EC00F2
:1024A200F0758F01750A00750900AE09AF0A74FF55
:1024B200C39F74019E402475B7A575B7F190004C77
:1024C20012001EE0FC90E60012001EECF0780A7486
:1024D2000126F6500418E436F650CF750A00750945
:1024E20000AE09AF0A74FFC39F74019E402475B702
:1024F200A575B7F190024C12001EE0FC90E80012A4
:10250200001EECF0780A740126F6500418E436F640
:1025120050CF750A00750900AE09AF0A74FFC39F58
:1025220074019E402475B7A575B7F190044C120052
:102532001EE0FC90EA0012001EECF0780A740126FC
:10254200F6500418E436F650CF750A00750900AE4D
:1025520009AF0A74FFC39F74019E402475B7A57525
:10256200B7F190064C12001EE0FC90EC0012001E27
:10257200ECF0780A740126F6500418E436F650CFCF
:10258200758F0075F51175B62075D940D2AF743AC2
:1025920090074CF022900786E0B4AA02800302263C
:1025A200D4C2AF75D90075B62275F522758F037541
:1025B200B7A575B7F1740090DE00F075B7A575B7D1
:1025C200F1740090E000F075B7A575B7F174009052
:1025D200E200F075B7A575B7F1740090E400F075EC
:1025E2008F01750A00750900AE09AF0A74FFC39F17
:1025F20074019E402475B7A575B7F190004C120086
:102602001EE0FC90DE0012001EECF0780A74012637
:10261200F6500418E436F650CF750A00750900AE7C
:1026220009AF0A74FFC39F74019E402475B7A57554
:10263200B7F190024C12001EE0FC90E00012001E66
:10264200ECF0780A740126F6500418E436F650CFFE
:10265200750A00750900AE09AF0A74FFC39F7401C1
:102662009E402475B7A575B7F190044C12001EE088
:10267200FC90E20012001EECF0780A740126F6507B
:102682000418E436F650CF750A00750900AE09AF9A
:102692000A74FFC39F74019E402475B7A575B7F1F4
:1026A20090064C12001EE0FC90E40012001EECF0BA
:1026B200780A740126F6500418E436F650CF758F66
:1026C2000075F51175B62075D940D2AF743A9007EE
:1026D2004CF022900786E0B4AA028003022812C2BC
:1026E200AF75D90075B62275F522758F0375B7A53A
:1026F20075B7F1740090D600F075B7A575B7F1748F
:102702000090D800F075B7A575B7F1740090DA00A3
:10271200F075B7A575B7F1740090DC00F0758F0104
:10272200750A00750900AE09AF0A74FFC39F7401F0
:102732009E402475B7A575B7F190004C12001EE0BB
:10274200FC90D60012001EECF0780A740126F650B6
:102752000418E436F650CF750A00750900AE09AFC9
:102762000A74FFC39F74019E402475B7A575B7F123
:1027720090024C12001EE0FC90D80012001EECF0F9
:10278200780A740126F6500418E436F650CF750A1A
:1027920000750900AE09AF0A74FFC39F74019E4021
:1027A2002475B7A575B7F190044C12001EE0FC9099
:1027B200DA0012001EECF0780A740126F6500418B2
:1027C200E436F650CF750A00750900AE09AF0A74F7
:1027D200FFC39F74019E402475B7A575B7F190069B
:1027E2004C12001EE0FC90DC0012001EECF0780A95
:1027F200740126F6500418E436F650CF758F007532
:10280200F51175B62075D940D2AF743A90074CF0E5
:1028120022C2AF75D90075F522750A00750900AE9E
:1028220009AF0A74FFC39F74019E401F90EE00120D
:10283200001EE493FC90004C12001EECF0780A7427
:102842000126F6500418E436F650D4750A007509CC
:1028520000AE09AF0A74FFC39F74019E401F90F03F
:102862000012001EE493FC90024C12001EECF07861
:102872000A740126F6500418E436F650D4750A009C
:10288200750900AE09AF0A74FFC39F74019E401F11
:1028920090F20012001EE493FC90044C12001EEC15
:1028A200F0780A740126F6500418E436F650D4750E
:1028B2000A00750900AE09AF0A74FFC39F74019E36
:1028C200401F90F40012001EE493FC90064C12008C
:1028D2001EECF0780A740126F6500418E436F6501D
:1028E200D475F51175D940D2AF22C2AF75D9007532
:1028F200F522750A00750900AE09AF0A74FFC39F7D
:1029020074019E401F90E60012001EE493FC9000AA
:102912004C12001EECF0780A740126F6500418E4FA
:1029220036F650D4750A00750900AE09AF0A74FF75
:10293200C39F74019E401F90E80012001EE493FCA6
:1029420090024C12001EECF0780A740126F6500434
:1029520018E436F650D4750A00750900AE09AF0ABC
:1029620074FFC39F74019E401F90EA0012001EE490
:1029720093FC90044C12001EECF0780A740126F6C7
:10298200500418E436F650D4750A00750900AE09F1
:10299200AF0A74FFC39F74019E401F90EC001200A7
:1029A2001EE493FC90064C12001EECF0780A7401AF
:1029B20026F6500418E436F650D475F51175D94050
:1029C200D2AF22C2AF75D90075F522750A0075091A
:1029D20000AE09AF0A74FFC39F74019E401F90DED0
:1029E2000012001EE493FC90004C12001EECF078E2
:1029F2000A740126F6500418E436F650D4750A001B
:102A0200750900AE09AF0A74FFC39F74019E401F8F
:102A120090E00012001EE493FC90024C12001EECA7
:102A2200F0780A740126F6500418E436F650D4758C
:102A32000A00750900AE09AF0A74FFC39F74019EB4
:102A4200401F90E20012001EE493FC90044C12001E
:102A52001EECF0780A740126F6500418E436F6509B
:102A6200D4750A00750900AE09AF0A74FFC39F74DA
:102A7200019E401F90E40012001EE493FC90064C5D
:102A820012001EECF0780A740126F6500418E4369F
:102A9200F650D475F51175D940D2AF22C2AF75D9AF
:102AA2000075F522750A00750900AE09AF0A74FFB8
:102AB200C39F74019E401F90D60012001EE493FC37
:102AC20090004C12001EECF0780A740126F65004B5
:102AD20018E436F650D4750A00750900AE09AF0A3B
:102AE20074FFC39F74019E401F90D80012001EE421
:102AF20093FC90024C12001EECF0780A740126F648
:102B0200500418E436F650D4750A00750900AE096F
:102B1200AF0A74FFC39F74019E401F90DA00120037
:102B22001EE493FC90044C12001EECF0780A74012F
:102B320026F6500418E436F650D4750A00750900DA
:102B4200AE09AF0A74FFC39F74019E401F90DC0060
:102B520012001EE493FC90064C12001EECF0780A60
:102B6200740126F6500418E436F650D475F5117542
:102B7200D940D2AF22E51464046006E59964FF608F
:102B8200028031A2104004D2108027E5146008743C
:102B9200E62514900023F0E513600874F0251390E5
:102BA2000023F0E514B4010280FE751400751300D1
:102BB200C2108002C210E5149034D8F82828737528
:102BC2001400E599B4FF03751301E599B4FE03758A
:102BD2001302E599B4FD03751303E599B4FC03757B
:102BE2001304E599B4FA03751305E599B4FB067568
:102BF20014011203B4E599B4F9067514041203B46E
:102C0200E599D394E54007E599C394F04002801614
:102C12008599157514027E017F00E515C394E612AD
:102C22003BB28E0D8F0E900784E4F0A3F0E599D3AA
:102C320094C44007E599C394E6400280288599151B
:102C420075140374E5C39515F50E750D00AE0DAF41
:102C52000E90353512002EE493F874019390078498
:102C6200C8F0A3C8F0D2990230EC900784E0FEA32A
:102C7200E0FFEFC39400EE94054009EFD394FFEE1A
:102C820094064013900784E0FEA3E0FF90004C12EC
:102C9200001EE599F0800385996C90078412000E5E
:102CA200900784E0FEA3E0FFEFB40106EEB4070252
:102CB2008003022EF990074CE0B43C028003022EFE
:102CC200F975FFA0A20AB35005A20BB34003022D6F
:102CD200ECC29C900078E090078AF0900055E0905A
:102CE200078BF0900060E090078CF0900061E0901C
:102CF200078DF0900072E090078EF090007AE090DD
:102D0200078FF090007BE0900790F090007EE090BB
:102D12000791F090007FE0900792F0900138E090E8
:102D22000793F0900139E0900794F090013AE09017
:102D32000795F090008EE0900796F090008FE0905B
:102D42000797F0900090E0900798F0900091E09043
:102D52000799F0900092E090079AF0900093E0902B
:102D6200079BF0900094E090079CF0900095E09013
:102D7200079DF0900097E090079EF0900098E090F9
:102D8200079FF0900099E09007A0F090009AE090E1
:102D920007A1F07400900080F012008F74AB9007CE
:0D2DA20086F012227074AA900786F0E558A2
:0634D800022BC1022C6C66
:102DAF009034F9F8282873801212231B800D1224F7
:0B2DBF0059800812259780031226D5CA
:0F34F900022DB6022DB8022DBD022DC2022DC725
:102DCA00900786E4F0900138E0700C900139E070C9
:102DDA000690013AE060028004C20A8002D20A0226
:102DEA002EEEC29C900076E0900787F090005CE09F
:102DFA00900788F090005DE0900789F0900078E0F5
:102E0A0090078AF0900055E090078BF0900060E000
:102E1A0090078CF0900061E090078DF0900072E0CE
:102E2A0090078EF090007AE090078FF090007BE098
:102E3A00900790F090007EE0900791F090007FE07C
:102E4A00900792F0900138E0900793F0900139E0F2
:102E5A00900794F090013AE0900795F090008EE088
:102E6A00900796F090008FE0900797F0900090E01E
:102E7A00900798F0900091E0900799F0900092E006
:102E8A0090079AF0900093E090079BF0900094E0EE
:102E9A0090079CF0900095E090079DF0900097E0D5
:102EAA0090079EF0900098E090079FF0900099E0BC
:102EBA009007A0F090009AE09007A1F074009000AB
:102ECA0080F074AB900786F012227074AA9007867D
:102EDA00F012231B1224591225971226D5D29C755B
:102EEA0099FB80FED29C7514007513007599FB023C
:102EFA0030EC900784E0FEA3E0FFEF4E7006859960
:102F0A0010750F00900784E0FEA3E0FF74016F4E76
:102F1A00701BAC0FAD10AA0DAB0EED2BFBEC3AFA01
:102F2A008A068B0790004C12001EE599F0900784E0
:102F3A0012000E900784E0FEA3E0FF74026F4E7049
:102F4A000C12008F8515997514007513000230EC68
:102F5A00900784E0FEA3E0FF90004C12001EE59962
:102F6A00F090078412000E900784E0FEA3E0FFAC05
:102F7A000DAD0E8F028E038C068D0790356D1200F3
:102F8A002EE493F9740193FEEAD39EEB99400985E6
:102F9A0015997514007513000230EC900784E0FE51
:102FAA00A3E0FF90004C12001EE599F090078412EE
:102FBA00000E900784E0FEA3E0FFEFB40006EEB433
:102FCA00010280030230EC75FFA090001CE0D3944C
:102FDA00C7400B90001CE0C394C8F516801A9000F5
:102FEA001CE0D39463400B90001CE0C39464F51674
:102FFA00800690001CE0F516E51675F002A4FFAEF7
:10300A00F08F6BEF90004C123BCAEFFCE0FDEC90A6
:10301A00004F123BCAEDFCE0FDEC2DB51602800311
:10302A000230DE0FEF90004C123BCAE56BFFE0FC6A
:10303A00EF900050123BCAECFFE0FCEFC39CB516C0
:10304A000280030230DEE56B90004E123BCAE56B4C
:10305A00FFE0FCEF900051123BCAECFFE0FCEF2CC2
:10306A00B51671E56B900052123BCAE0C3951690F3
:10307A00079BF0E56B900053123BCAE0C39516908C
:10308A00079CF0E56B900056123BCAE0C395169078
:10309A00079DF0E56B900057123BCAE0C395169066
:1030AA00079EF0E56B900058123BCAE0C395169054
:1030BA00079FF0E56B900059123BCAE0C395169042
:1030CA0007A0F01221E67599F975186475170012B0
:1030DA0021A280FE7599FF7518647517001221A246
:0230EA0080FE66
:0934DE00022EFC022F5A022FA558
:1030EC0022E5139034E7F828287302322D900784D8
:1030FC00E0FEA3E0FF90001212001EE0F59990078D
:10310C008412000E900784E0FEA3E0FF74116F4E52
:10311C00700375130002322D85629902322D9007CF
:10312C0084E0FEA3E0FF90004C12001EE0F599EF46
:10313C00B40107EEB4070375130090078412000E58
:07314C0002322D900785E01F
:0F34E7000230F60230F902312402312A02314F4D
:10315300903508F8282873852499023222852A9904
:10316300023222854499023222854799023222850E
:103173005199023222856099023222855699023290
:1031830022855899023222756E00900067E070061E
:10319300900066E060028016A2A44006E56E440437
:1031A300F56EA2A54006E56E4402F56E801A900006
:1031B3004AE0B40106E56E4410F56E900049E0B4B0
:1031C3000106E56E4420F56EA207B34006E56E44A2
:1031D30001F56EA209B34006E56E4408F56E856EEF
:1031E30099803CA211B340077599FAC2118017A2C6
:1031F3000CB3400575990F800B900023E0F599906F
:103203000023E4F0C20C80178542998012854B9904
:0F321300800D85469980087599FC80037513001E
:1035080002315A02316002316602316C02317202B4
:10351800317802317E02318402318A0231E6023288
:0D3528000B02321002321502321A02321F5D
:0B32220090078412000E800312004889
:0334F60002322A75
:10322D0022900069E0B40103852411900069E0B497
:10323D000203852A11900069E0B4030385441190BF
:10324D000069E0B40403854711900069E0B40503FB
:10325D00855111900069E0B40603855611900069FF
:10326D00E0B4070385581190006AE0FE90006BE012
:10327D00C39E5003023304900069E0D39404402CA4
:10328D0090006AE0D39511500990006BE0C3951141
:10329D0050028002D20090006AE0D395115009903F
:1032AD00006BE0C395115002C2008049900069E0A7
:1032BD00B4041890006BE0C395115002D200900039
:1032CD006AE0D395114002C200802A90006AE0C3E3
:1032DD009511500990006BE0D3951150028002D2E8
:1032ED000090006AE0D39511500990006BE0C395F2
:1032FD00115002C200807E900069E0D39404402CEE
:10330D0090006AE0C39511400990006BE0D39511D0
:10331D0040028002C20090006AE0C39511400990FE
:10332D00006BE0D395114002D2008049900069E016
:10333D00B4041890006AE0C395115002C2009000C9
:10334D006BE0D395114002D200802A90006AE0C351
:10335D009511400990006BE0D395114002D2009079
:10336D00006AE0D39511400990006BE0C3951140C0
:10337D00028002C2002290006CE0B401038524118A
:10338D0090006CE0B40203852A1190006CE0B40348
:10339D000385441190006CE0B4040385471190003F
:1033AD006CE0B4050385511190006CE0B406038503
:1033BD00561190006CE0B4070385581190006DE034
:1033CD00FE90006EE0C39E500302345990006CE0F5
:1033DD00D39404402C90006DE0D3951150099000CA
:1033ED006EE0C3951150028002D20290006DE0D3C1
:1033FD009511500990006EE0C395115002C20280E4
:10340D004990006CE0B4041890006EE0C395115023
:10341D0002D20290006DE0D395114002C202802AC3
:10342D0090006DE0C39511500990006EE0D3951199
:10343D0050028002D20290006DE0D3951150099098
:10344D00006EE0C395115002C202807E90006CE0C8
:10345D00D39404402C90006DE0C395114009900069
:10346D006EE0D3951140028002C20290006DE0C360
:10347D009511400990006EE0D395114002D2028063
:10348D004990006CE0B4041890006DE0C3951150A4
:10349D0002C20290006EE0D395114002D202802A42
:1034AD0090006DE0C39511400990006EE0D3951129
:1034BD004002D20290006DE0D39511400990006E4C
:0B34CD00E0C3951140028002C2022201
:093BCA002582F5825002058322D8
:10002E00EF2F500205832582F582E5833E2EF58360
:01003E00229F
:08000300C3EF9DFFEE9CFE22FD
:08003F000806B60002180622B3
:0D000E00A3E004F07006123BC0E004F022F5
:083BDC000816B6FF02181622BC
:0E3BA400048007C3CE13CECF13CFD5E0F62298
:103A5200BC000FBE0008ED8FF084FFADF022E4FE43
:103A6200FF22BE000DEF60FE54F0606F20E70302FC
:103A72003B08EAC0E0EBC0E078017A0075F001EEA5
:103A820020E710EF25E0FFEE33FE0AC5F023C5F074
:103A920030E7F0EA5407F9096A7A007B006001080E
:103AA200C3EC9E40167004ED9F4010ED9FFDEC9E0E
:103AB200FCE5F0CA4ACA03F5F08005E5F003F5F02B
:103AC200C3EE13FEEF13FFD9D77908CACBCAD8D0F9
:103AD200EAFEEBFFD0E0FBD0E0FA22EC8FF084FCB0
:103AE200ED54F045F0C48FF084FEEDC454F045F07F
:103AF200C48FF084FDEEC4FE54F02DFFEE540F3C53
:103B0200FEADF07C0022790078008FF0EC7E082078
:103B1200E70DC3CD33CD33C933C9C833C8DEF08412
:103B220049F9E5F08FF0BE00E6FD7C00E9FFE8FE12
:013B32002270
:0E3BB200F88FF0A4FFE5F0CE88F0A42EFE22DE
:103B8400600D782B023B8E007830D8FED5E0F82209
:103B9400EEC0E07E00123A52EFFDEEFCD0E0FE22D1
:03000B00023B3382
:03001B00023B4E57
:03002B00023B692C
:03000000023BD3ED
:093BD30075817275D000020581B4
:0B001E00E5822FF582E5833EF583228A
:0A3BC0000582D582021583158222CA
:103B3300C0E0C0F0C083C082C0D075D0001205764B
:103B4300D0D0D082D083D0F0D0E032C0E0C0F0C07B
:103B530083C082C0D075D000120579D0D0D082D076
:103B630083D0F0D0E032C0E0C0F0C083C082C0D0C8
:103B730075D00012057CD0D0D082D083D0F0D0E0B5
:013B8300320F
:00000001FF
